:100000000C9463140C9480140C9474170C94801446
:100010000C9480140C94A1170C9480140C948014EC
:100020000C9480140C9480140C9480140C948F15F0
:100030000C9480140C9480140C949E150C948014D1
:100040000C9480140C9480140C9480140C948014E0
:100050000C9480140C9480140C9480140C948014D0
:100060000C9480140C9480140A00080402010C06FD
:1000700083016EB7DB0DEFF7FB0DFFFFFF0F5EAFE8
:10008000D70BDD6AB70AFFFFFF0F0000000000007A
:100090000000290081402000120281028008240013
:1000A000026150002010080402814000241009045D
:1000B00040201008241088000800000044120800A6
:1000C00008040000042081000804020000009100E0
:1000D0000804020104014100201408050401410044
:1000E000402410090003C0004820120820114804D1
:1000F00008068201040141004022900824114904AD
:10010000402010080003C000040001000283C0006A
:1001100024100904128944028542A1000281400092
:100120008140200002814000040281000804000197
:1001300044228100000010090800814020000804CA
:1001400002011008040204028100814020002010F6
:1001500008044020100802814000100008008008B8
:100160000000000000001101000000000022020059
:1001700000000000440000040000000000404404AF
:10018000000000008088080000000000111100003D
:100190000000000022002002000000000D00880086
:1001A0002200014400014008100210200408200829
:1001B000080201414000828020000011400422809A
:1001C0000800002280084400110008040201040114
:1001D00041001800814020000000000010080402C7
:1001E0000000000002814000000000002010080410
:1001F0000000000004028100000000004020100800
:100200000000000008040201000000004020100867
:10021000000000000402810000000000201008041B
:1002200000000000028140000000000010080402ED
:10023000000000001D00080002000020000800026D
:1002400080002000080002800000001000028000F2
:1002500020000008000202800000200008000002C8
:1002600080000020000808000200080402010000CD
:100270000000000400014000100004000100001014
:1002800000040001400010000400014000001000C4
:1002900004000001400000100004040001004000C0
:1002A00010000004000108040201380008000200E8
:1002B0000000000000200008000000000002800094
:1002C0000000000020000800000000000280000084
:1002D000000000000010000200000000800020006C
:1002E0000000000000080002000000000280000082
:1002F0000000000020000800000000000002800054
:1003000000000000002000080000000008000200BB
:1003100000000000080402010000000000040001C9
:100320000000000040001000000000000400010078
:100330000000000000100004000000000001400068
:100340000000000010000400000000000140000058
:100350000000000010000400000000000001400048
:100360000000000000100004000000000400010074
:100370000000000040001000000000000004000128
:100380000000000008040201000000001900A9524A
:10039000AA0400000000A952AA0400000000A9520B
:1003A000AA040000000056AD550B00000000A95241
:1003B000AA0400000000A952AA040000000056ADE3
:1003C000550B00000000A952AA040000000056AD21
:1003D000550B00000000A952AA0400000000A95219
:1003E000AA040000000056AD550B00000000A95201
:1003F000AA049100500014000000000050001400F6
:10040000200008000000000020000800000000009C
:10041000000140000000000000014000000000005A
:100420008002A000000000008002A0000000000088
:100430000028000A00000000001000040000000076
:100440000010000400000000028000000280000094
:100450000000000005400100000000000540010010
:10046000000000000804020100000000080402016E
:10047000000000000804020100000000080402015E
:10048000000000000804020100000000080402014E
:10049000000000004422910800000000442291085E
:1004A000000000000804020100000000080402012E
:1004B000000000004422910800000000442291083E
:1004C000080402010000000008040201000000000E
:1004D000442291080000000044229108000000001E
:1004E000229148040000000022914804000000000E
:1004F00044229108000000004422910808040201EF
:1005000000000000080402010000000044229108DD
:1005100000000000442291080000000022914804DD
:1005200000000000229148040000000091482402CD
:1005300000000000914824020000000022914804BD
:1005400000000000229148040000000044229108AD
:10055000000000004422910800000000080402018D
:1005600000000000080402010000000004028100F5
:100570000000000004028100000000000281400031
:1005800000000000028140000000000081402000C7
:10059000000000008140200000000000100804025C
:1005A00000000000100804020000000020100804F1
:1005B0000000000020100804000000000402810078
:1005C000000000000402810000000000402010082C
:1005D0000000000040201008000000000804020194
:1005E00000000000080402010000000008040201ED
:1005F00000000000914824020000000008040201ED
:1006000000000000080402010000000091482402DC
:1006100091482402000000000804020100000000CC
:100620000C800100000000000540010000000000F7
:100630000540010000000000440008040201000021
:10064000000008040201000000000804020100008C
:10065000000008040201000000000804020100007C
:10066000000091482402229148044422910800008D
:10067000000008040201000000000804020100005C
:10068000000091482402229148044422910800006D
:100690000000080402010000000008040201914863
:1006A0002402000000009148240200000000229172
:1006B0004804000000002291480400000000442289
:1006C0009108000000004422910800000000080486
:1006D000020144229108229148049148240208040E
:1006E000020144229108229148049148240200000A
:1006F00000009148240222914804442291080000FD
:100700000000080402010000000044229108229128
:10071000480400000000000000009148240200008E
:1007200000000000000008040201000000000000BA
:10073000000000000000FFFFFF0F000000000000AD
:100740000000080402010000000049008542A100E9
:100750000000000081402000000000008542A10050
:100760000000000081402000000000000402810021
:1007700000000000040281000000000030180C0698
:10078000000000000402810000000000040281005B
:1007900000000000040281000000000030180C0678
:1007A00000000000040281000000000012894402E1
:1007B0000000000081402000000000001289440277
:1007C0008140200030180C06040281001289440286
:1007D00008040201100804020402810032994C0648
:1007E00004028100128944020000000022914804A2
:1007F0000000000012894402000000002291480419
:1008000000000000100804020000000022914804CB
:1008100000000000040281000000000062B0180C1B
:100820000000000022914804000000005028140A33
:10083000000000008542A10000000000128944026F
:10084000000000008542A100000000002291480441
:100850008D46A30172B95C0E8D46A3015028140A7F
:100860008D46A3015028140A8D46A3010000000004
:100870005F0091482402000000009148240200001B
:10088000000091482402000000009148240200006A
:10089000000091482402000000002291480400005A
:1008A000000022914804000000002291480400004A
:1008B000000022914804000000002291480400003A
:1008C000000044229108000000004422910800002A
:1008D000000044229108000000004422910800001A
:1008E00000000804020100000000080402010000EA
:1008F00000004422910800000000442291080000FA
:1009000000002291480400000000229148040000E9
:100910000000914824029148240200000000229126
:100920004804229148040000000044229108442217
:10093000910800000000080402014422910822915D
:1009400048049148240200000000914824022291AA
:10095000480491482402229148044422910822919B
:10096000480491482402000000009148240222918A
:10097000480444229108080402019148240222916B
:10098000480444229108080402019148240222915B
:1009900048044422910808040201000000000804F1
:1009A0000201000000000804020100000000080429
:1009B000020100000000FFFFFF0F0000000008041C
:1009C000020100000000080402010000000091483C
:1009D00024020000000008040201000000000804D6
:1009E0000201000000009148240200000000A30062
:1009F0008FC7E301000000008FC7E3010000000083
:100A00008FC7E301000000008FC7E3010000000072
:100A10008FC7E301000000008FC7E3010000000062
:100A20008FC7E301000000008FC7E3010000000052
:100A30008FC7E3010000000070381C0E00000000AA
:100A400070381C0E000000008FC7E301000000009A
:100A50008FC7E3010000000070381C0E000000008A
:100A600070381C0E000000008FC7E301000000007A
:100A70008FC7E3010000000070381C0E000000006A
:100A800070381C0E000000008FC7E301000000005A
:100A90008FC7E3010000000070381C0E000000004A
:100AA00070381C0E000000008FC7E301000000003A
:100AB00070381C0E000000008FC7E301000000002A
:100AC00070381C0E000000008FC7E301000000001A
:100AD00070381C0E000000008FC7E301000000000A
:100AE00070381C0E000000008FC7E30170381C0E28
:100AF0008FC7E30170381C0E8FC7E30170381C0EDE
:100B00008FC7E30170381C0E8FC7E30170381C0ECD
:100B10008FC7E30170381C0E0000000070381C0EF7
:100B20000000000070381C0E0000000070381C0E21
:100B30000000000070381C0E0000000070381C0E11
:100B40000000000070381C0E0000000070381C0E01
:100B50000000000070381C0E0000000070381C0EF1
:100B60000000000070381C0E0000000070381C0EE1
:100B70000000000070381C0E000000008FC7E30169
:100B8000000000008FC7E3010000000070381C0E59
:100B90000000000070381C0E000000008FC7E30149
:100BA000000000008FC7E3010000000070381C0E39
:100BB0000000000070381C0E000000008FC7E30129
:100BC000000000008FC7E3010000000070381C0E19
:100BD0000000000070381C0E000000008FC7E30109
:100BE000000000008FC7E3010000000070381C0EF9
:100BF000000000008FC7E3010000000070381C0EE9
:100C0000000000008FC7E3010000000070381C0ED8
:100C1000000000008FC7E3010000000070381C0EC8
:100C2000000000008FC7E3010000000070381C0EB8
:100C30008FC7E30170381C0E8FC7E30170381C0E9C
:100C40008FC7E30170381C0E8FC7E30170381C0E8C
:100C50008FC7E30170381C0E8FC7E30170381C0E7C
:100C60008FC7E30170381C0E8FC7E30170381C0E6C
:100C70008FC7E30170381C0E00000000390000002F
:100C80002000000004000040000000080000800078
:100C90000000100000000100000000000002000041
:100CA000400000000800008000000010000000016B
:100CB000000020000000020000000000000400000E
:100CC0008000000010000000010000200000000271
:100CD00000004000000004000000000000080000C8
:100CE00000010000020000040000080000000000F5
:100CF00000010000020000040000080000000000E5
:100D0000000800008000000010000000010000202A
:100D1000000000020000400000000400000000008D
:100D200000080000800000000800008000000010A3
:100D30000000000100002000000002000000000090
:100D40000004000040000000040000400000000813
:100D50000000800000001000000001000000000002
:100D6000000207000804020140201008040281006C
:100D70002010080402814000100804028140200075
:100D80001B008000200000014000000280000004E1
:100D90000001080002000020000800100004000804
:100DA00000020010000400200008000400010800F8
:100DB00002000400010002800000014000000280E7
:100DC00000000400010008000200400010002000A4
:100DD0000800100004002000080040001000080077
:100DE0000200000400010002800000014000160023
:100DF00070381C0E0000000087C3E10000000000F6
:100E000008040201000000004422910800000000D4
:100E100022914804000000009148240200000000D4
:100E200091482402000000002291480400000000C4
:100E30004422910800000000080402010804020195
:100E4000080402010000000036000100000010004C
:100E5000000080000000000800000040000000804A
:100E60000400000021000000020209000200090441
:100E70000201090682010943C2008947E20100001C
:100E80000000442291080000000022914804000064
:100E90000000914824020800000000040000000047
:100EA0000200000000010400000000020000000039
:100EB000010000008000020000002000000000018E
:100EC000000000100000008000000000080000008A
:100ED00040000000000402000000010000001000BB
:100EE0000002800020000008040000400000080408
:100EF00002014422910822914804914824020804E6
:100F000002014422910822914804914824020804D5
:100F100002019148240208040201914824020000C1
:100F200000002D0008060001480400010C04000127
:100F300008040009080480010804100108040101E4
:100F40000824000108060001480400010C04000107
:100F500008040009080480010804100108040101C4
:100F60000824000108060001480400010C040001E7
:100F700008040009080480010804100108040101A4
:100F80000824000108060001480400010C040001C7
:100F90000804000908048001080410010804010184
:100FA0000804020104028100028140008140200007
:100FB000814020008140200010080402028140008E
:100FC00020100804040281004020100808040201D7
:100FD00008040101082400012A000000200000008C
:100FE0004000000080000000000108000000040034
:100FF00000000200000001000000000000000000EE
:10100000000000000000800000000001000000025D
:101010000000000400000000020000000100008049
:101020000000004000000000000000000000000080
:101030000000000004000000080000001000000094
:101040000001000000080000000400000002000091
:101050000000000000000000000010000000200060
:10106000000040000000000400000020000000100C
:101070000000000800000000000000000000000068
:101080000000110001000000120000022400000412
:101090004000000808040001080280000801400028
:1010A00088002000080140000802800008040001B8
:1010B000002012000010090000880400004804000D
:1010C00080002000100000020D000100000002005E
:1010D0000000040000004000000820000004100090
:1010E000000280002000000804000010080000201A
:1010F00010000000010000800000004000003700E8
:101100000E8003000E8003000E8003000E8003009B
:101110000E800300700D460F700D460F700D460FC8
:10112000700D460F700D460F220E8405220E8405A9
:10113000220E8405220E8405220E84050296880460
:10114000029688040296880402968804029688040F
:101150000284880502848805028488050284880543
:10116000028488050000000000000000000000006C
:101170000000000000000000183E860F183E860F99
:10118000183E860F183E860F183E860F229148049F
:101190002291480422914804229148042291480453
:1011A0002E9103002E9103002E9103002E91030037
:1011B0002E91030002848805028488050284880534
:1011C00002848805028488050000000000000000F9
:1011D00000000000000000000000000042000000CD
:1011E00064000000640000004C000000C800000023
:1011F00098000000900100001201000402010804A0
:1012000000014804000040060000600200002003C6
:1012100000003001000090010000900100008009F2
:101220000000001900000058000000D0000000C0BD
:10123000040000800C0000004C000000640000006E
:1012400060020000400601000006030000040600E2
:1012500000040400000C0C00000808000009080449
:1012600000010004020100240200002003000030FD
:101270000100009001000098000000C8000000C8B4
:10128000000000C0040000800C0000800900000085
:10129000190000001300002003000030010000329C
:1012A00000000013000020030000300100003200A5
:1012B00000006200000060020000400600000026FE
:1012C000000040060000480400004C0000000C0034
:1012D00000080400000C0000800C0000C0040000A6
:1012E000C80000004C004E00001000040010000474
:1012F00000100004000000000000000000000000DA
:101300002000080020000800200008000000000065
:101310000000000002814000028140000281400084
:10132000000000000000000000000000100804029F
:101330001008040210080402000000000000000071
:10134000000000008000000000010000000200001A
:1013500000040000000000010000800000004000C8
:10136000000020000000000000000000000000005D
:10137000000000000000000000000000010000006C
:10138000020000000400000008000000000002004D
:10139000000001000080000000400000000000008C
:1013A000000000000000000000000000000000003D
:1013B00000000000000800000010000000200000F5
:1013C0000004020008000001000000080000000402
:1013D000000000020000000000000000000000000B
:1013E00000000000000000000000040000000800F1
:1013F000000010000000020108040000400000008E
:1014000020000000100000000000000000000000AC
:1014100000000000000000000000000000000000CC
:101420002E00080000000004000000000200000080
:10143000000108000000000400000002000000019C
:101440000000800000000008000000100000000103
:101450000000000200000020000000000100000069
:10146000020008000000040000000200000001006B
:101470000000000000020000000400004000000026
:1014800080000000000800000001000010000000C3
:101490000800000004000040000000800000000080
:1014A000010000000200080000000400000002002B
:1014B0000000010000001000000080000000000893
:1014C000000000100000008000000000010000206B
:1014D000000000040000080000002A000000540082
:1014E0000000A800000050020100A000100040020F
:1014F0008100200010080002814000001008040054
:1015000080402000008140000002080402044000E6
:101510002000000502018000201040000081200012
:1015200000420002018400001000010180008200DE
:1015300008084000041020000220040001400100BF
:1015400002081000201080000021400080002200CE
:10155000080140002400080042800000094000000B
:101560001008000180108000002840000044200086
:101570000880000200000105000082080000500100
:101580000000A80042000000080000000100000068
:10159000020008000000000400000020000000100D
:1015A0000000000100008000000000080000004072
:1015B000000000800000000001000000100000009A
:1015C000080000000400004000000080000000004F
:1015D00001000000100000000200002000000002D6
:1015E0000000000400000000000100008000000076
:1015F000400000000800000004000000200000007F
:101600004000000080000000000800000001080009
:1016100000000004000000020000000100000010B3
:101620000000002000000002000000010000200077
:101630000000100000000100000002000000200077
:10164000000040000000080000000000000800004A
:101650000004000000020000200000004000000024
:101660000004020000000400000008000000000068
:10167000020000000100002000000010000000082F
:1016800000000040000000800000000004002F0067
:101690000000C0080000E001000060020000200619
:1016A0000000200E0800000C4800000C680000003C
:1016B0007800000031000000330000000700000047
:1016C00047000000440200004403000080030000C3
:1016D00090030000B0000000F00000006004000073
:1016E0006004020000040201080402010804000171
:1016F00008040201000403000084030000C001008C
:1017000000C801000058000000780000003200000E
:1017100000330000200300006003000068000000A8
:10172000680000010800100108001101008011008C
:1017300000C0110000C0040000C00C0000001C002C
:1017400000001C0100009001000090094100000011
:1017500000020008000010000000000004008000EB
:1017600000000000200001000000004000002000F8
:1017700008000010000400028000040001000200C4
:1017800000002000000000010000001000000080A8
:101790000000001000000001000020000000020016
:1017A000000000000004000040000000080000806D
:1017B00000000000080000004000000000040200DB
:1017C0000000000000000000000000000000000019
:1017D0000000000000008140200010080402028187
:1017E0004000201008040402810040201008080472
:1017F00002010402810002814000814020000804AF
:1018000002018140200008040201000000000000E5
:1018100000000804020100000000000000000804AD
:10182000020100000000080402010000000008049A
:1018300002010000000044229108000000002291F3
:10184000480400000000914824020000000000004D
:1018500000001D0000002000000000020200000047
:101860002000000000020000002000000000020034
:101870000100000010000000000100000010000046
:101880000000010000001000000000010000000046
:101890008000000000080000008000000000080038
:1018A0000000800000000008080000000040000068
:1018B00000000400000040000000000404000000DC
:1018C0004000000000040000330000400000000859
:1018D0000000800000000001000000020000000481
:1018E0000000000000010000800000004000000037
:1018F0002000000004000040000000800000000004
:1019000001000000020000000001080000000004C7
:1019100000000000020000000001080000000004B8
:1019200000000000020000000001080000000004A8
:101930000000000002000000000108000000040098
:101940000000020000000100000000000002010091
:1019500000040000000A090000044000000A2800FA
:10196000000450000008290000005200000025007B
:1019700000001A000000050002000A0001000480B7
:1019800002000840010000C0020000C0010000C0C9
:101990000000004000002100743C1C0F743C1C0F30
:1019A000743C1C0F743C1C0F743C1C0F743C1C0DCD
:1019B000643C1C0D643C1C0D643C1C09443C1C092B
:1019C000003C1C09003C1C01003C1C0000381C00B1
:1019D00000380C0000180C000018040000080C006F
:1019E00000080400000004000000000000080400DB
:1019F00000080C000008440000088C00001A4C008D
:101A0000000C0C08400C0400200C040400124800D8
:101A10000021900040000009200000043B0000402D
:101A200024000040280000403000008042014000B7
:101A30008100202000081402000002010000810043
:101A400000001000000020000000C10000000A0596
:101A5000000004021000002008080000850000803B
:101A600040000040200000080002001000040402B2
:101A7000810040001000000400000000020000008F
:101A80000001080000000004000000000200000047
:101A90000001000000080400800402004002010070
:101AA000200201002004010020080A004001040473
:101AB00082004020100000120100008900008048D0
:101AC00000008050000000A1000000060300480054
:101AD0001001040080040200400201002002000006
:101AE00000000000000000000000000000000000F6
:101AF00000000000000000000000000000000000E6
:101B0000000000000000000000002A0004000100A6
:101B1000400010000002800040001000040001009E
:101B2000040001000400010004000100002000087E
:101B300000028000002000080400010004000100F1
:101B400004000100040001004000100000028000B9
:101B5000400010000400010040001000000280005E
:101B6000400010000400010040001000000280004E
:101B7000400010000400010040001000000280003E
:101B8000002000080400010000200008000280007E
:101B900000200008040001002290080411480402FB
:101BA000229008041148040222914804442291081A
:101BB000080402012B00040210002000010402109E
:101BC00040008000040210402000011008000220A4
:101BD0001000040400014800000820000204100066
:101BE0000102808020000041400000900800004871
:101BF0000400009148000020110000229000000025
:101C0000C0000003000090002002200140044002B8
:101C100080080804000144000008220000041100AC
:101C200000022200000444000008040280000402B4
:101C3000100004021000040210000402100004024C
:101C4000100004021000040201000402100004024B
:101C500080000402100004020100040210000402CB
:101C60008000210080002000100000020100000020
:101C7000000140002000000402000000000280007B
:101C800040000008040000000004000108000000FB
:101C900000080400001008000020100000000200EE
:101CA00000040001400000082000000410000002B1
:101CB00080002000000804000040000000800000B8
:101CC000001008000001400020000004400000084F
:101CD000000400010000020000000100008000007C
:101CE00000400000000804001C010140000003C087
:101CF0000000068001000420010800228008400244
:101D000090004400110004200108002280084002D5
:101D100090004800120008040201080002000000C0
:101D20000000000000000000000000000000482447
:101D300012096C369B0D7EBFDF0FFFFFFF0FF57A98
:101D4000BD0EFFFFFF0FFFFFFF0FFFFFFF0FF7FBB2
:101D5000FD0EB3D96C06994C260308040201241227
:101D600089042412890412894402128944028140A0
:101D70002000814020000000000000000000000062
:101D80000000000000000000000000000000000053
:101D900000000000000000080000001800000038EB
:101DA0000000003002000020120000001A000000B5
:101DB0001C0000000C0000000400000000001000E7
:101DC00000003000000070000000680000004800C3
:101DD00000080800000C0000000E000000060000D3
:101DE00000020000000000000000000000000100F0
:101DF00000000100000001000000010000000100DF
:101E000000000100000001000000010000000300CC
:101E100000000300000003000000030000000300B6
:101E2000000003000000070000000700000007009A
:101E3000000007000000070000000F0000000F0076
:101E400000000F00000007000200030001000180F5
:101E50000000004000000140000003400000074077
:101E60000000074000000340000001400000014066
:101E7000000003400000014000000140000001405C
:101E80000000004000000040000000400000004052
:101E90000000004000000040000000400000004042
:101EA0000000004000000040000000400000004032
:101EB0000000004000000040000000400000004022
:101EC0000000004000000040000000400000004012
:101ED0000000004000000040000000400000004002
:101EE0000000004000000080000000800000008032
:101EF00000000080000000800000008000000080E2
:101F000000000080000000800000008000000080D1
:101F100000000080000000800000000001000000C0
:101F200001000000010000000100000001000000AD
:101F3000010000000100000001000000010000009D
:101F4000010000000100000001000000010000008D
:101F5000010000000100000001000000020000007C
:101F60000200000002000000020000000200000069
:101F70000200000002000000020000000200000059
:101F80000200000002000000020000000200000049
:101F90000200000002000800000008000000080025
:101FA0000000080000000800000008000000080011
:101FB0000000080000000800000008000000080001
:101FC00000000800000008000000080000000804ED
:101FD00002010804020108040201080402010804C5
:101FE00002010804020108040201080402010804B5
:101FF000020108040201080402014824120908042D
:10200000020108040201482412090804020108041C
:102010000201080402010804020108040201080484
:102020000201080402014824120928140A05582C48
:10203000160B28140A05582C160B28140A05582CC0
:10204000160B28140A05582C160B28140A05582CB0
:10205000160B28140A05582C160B28140A05582CA0
:10206000160B28140A05582C160B28140A05582C90
:10207000160B28140A05582C160B28140A05582C80
:10208000160B28140A05582C160B28140A05582C70
:10209000160B28140A05582C160B28140A05582C60
:1020A000160B28140A05582C160B28140A05582C50
:1020B000160B28140A05D96C360BA9542A055AADFB
:1020C000560B2A954A055C2E970B2C168B05582C1F
:1020D000160BA9542A05D96C360B2A954A055AAD18
:1020E000560B2C168B055C2E970B28140A05D96C01
:1020F000360BA9542A055AAD560B2A954A055C2E73
:10210000970B2C168B05582C160BA9542A05D96C45
:10211000360B2A954A055AAD560B2C168B055C2EAC
:10212000970B28140A05D96C360BA9542A055AAD09
:10213000560B2A954A055C2E970B2C168B05582CAE
:10214000160BA9542A05D96C360B2A954A055AADA7
:10215000560B2C168B055C2E970B0100FFFFFF0F13
:10216000150010080402201008044020100808047C
:102170000201040281000281400081402000100819
:102180000402028140002010080404028100402063
:10219000100808040201040281000281400081400D
:1021A0002000028140000402810008040201402056
:1021B00010082010080408000000000200002000A1
:1021C0000000040000400000000800008000000043
:1021D00010000000010000001C00010000000200CF
:1021E000000004000000080402010000010000805B
:1021F000000000400000000020000000400000003F
:1022000080000804020100020000000100008000BC
:10221000000000080000001000000020000008047A
:10222000020100000008000000040000000210008D
:10223000000020000000400000000804020100002F
:10224000100000000800000004003A000100000037
:1022500010000000800000000008000000400000A6
:10226000000004000000200000004000000080008A
:102270000000000100040000000200000001000056
:1022800020000000020000000000000400004000E8
:1022900000000800008000000000010000000200B3
:1022A00008000000040000004000000000020000E0
:1022B000002000000000010000001000000080006D
:1022C0000000000100040000000002000000000106
:1022D00008000000000400000000020000000001EF
:1022E00008000000000400000002000000010000DF
:1022F000800000001000000001000000000000024B
:102300000000200000000400004000000008000061
:102310008000000000010000000200000004000036
:1023200000000001000080000000400000002000CC
:10233000000000020C00028140008400210008011E
:1023400042000402810002840001014280000281F7
:102350004000840021000801420004028100028440
:102360000001014280001C0001000000020000008A
:1023700004000000080402010000010000800000C9
:10238000004000000000200000004000000080002D
:1023900008040201000200000001000080000000AB
:1023A00000080000001000000020000008040201E6
:1023B00000000008000000040000000210000000FF
:1023C000200000004000000008040201000010008E
:1023D00000000800000004002300814020001008D5
:1023E0000402028140002010080404028100402001
:1023F000100808040201000280000400010000101F
:1024000000042000080000014000028000001000CD
:10241000040000080002014000008000200001408C
:102420000000000800021000040000080002028002
:102430000000000140000010000404000100000240
:102440008000400010000020000800100004200060
:102450000800028000000001400000080002100097
:1024600004008000200012008400080000810008A1
:10247000004200040020040201002200100040017C
:1024800088008000000C00080412000000210008F1
:10249000800001041000100220000804400004081D
:1024A000000288000081400020402000120040000F
:1024B000500088000201080102010802020108041C
:1024C00002010404810002844000014420000284CF
:1024D000400004048100080402010802020108010E
:1024E000020188000201080002030800020508003A
:1024F00002094020100820100804100804020208F5
:102500000402000804060008C40000081C0000C8FB
:10251000010000380000700000000700000000000B
:10252000000E0000E00000003C0000C02100003868
:102530002000800320007000200007002000000021
:10254000200E0000E0000000040E074000007008AC
:102550000000800300007008000007400000000039
:10256000040E0000E0000000040E074000007008A8
:10257000000080030000202800000240010000004D
:1025800014040000E00000001404024001002028B0
:10259000000080030000202800000240010000002D
:1025A00014040000E00000003C0201C021021138C8
:1025B0002002910320020138200200C02102000005
:1025C0003C000000E0000000900E0300910070202D
:1025D000910080239100702091000700910000007D
:1025E000900E0000E0000000C0010004800108001F
:1025F0000201330004000000000000080000800019
:102600000000100000000100002000000002000097
:102610004000000004000000020000000100000073
:10262000000000080000000400000002000080001C
:102630000000400000002000000010000000080022
:1026400000000400000001000080000000400000C5
:102650000020000000100000000800000002000040
:102660000001000080000000400000002000000089
:102670001000000002000000000000020000400006
:1026800000000400008000000008000000010000BD
:10269000100000000200000004000000080000001C
:1026A0000000020000000100008000000040000067
:1026B000914824022291480444229108080402010E
:1026C0003600010000001000000280002000000819
:1026D000040000400000008000000010080000011D
:1026E0004000200000040200000001000000020081
:1026F00000000400000040000008000280000020EC
:102700001000000001000080000000400000008078
:1027100000000000010000000200000400010800A9
:1027200000000400000002000000010000000200A0
:102730000000040000000800000000040001000286
:1027400080000001400080002000000140000002E5
:102750008000000400010000020000000100008071
:1027600000000040000000800000000001000000A8
:10277000020008040201402010082010080410087C
:10278000040220100804402010080804020104007C
:10279000000002000000000000001400018480001E
:1027A000000000001004100400000000A000020857
:1027B00000000000088810000000000000448800AD
:1027C0000000000000044408000000004000220453
:1027D000000000004200020200000000210202008E
:1027E0000000000010210001000000003600402021
:1027F000100804028100201008040402810008046B
:102800000201402010080402810020100804028107
:102810004000201008044020100808040201402055
:102820001008040281002010080402814000814049
:10283000200010080402800020000008000201406F
:102840000000100004000000200000000002010051
:1028500000001000000080000000000800000040A0
:102860000000000004000000200000000002010041
:102870000000100000008000000000080000004080
:102880000000008804000010090000201000000073
:1028900002000004000108000000400000082400BD
:1028A000000412000002010000001100000291006B
:1028B00020029108240291482402229148044422D3
:1028C00091080804020111241FBECFEFD4E0DEBF3F
:1028D000CDBF11E0A0E0B1E0EAEDFBE302C005905E
:1028E0000D92AC30B107D9F711E0ACE0B1E001C016
:1028F0001D92AA3AB107E1F70E943E1C0C94EB1D11
:102900000C9400009C018091A201841710F4409166
:10291000A20180E00AC060FF05C0E82FF0E0E85D9A
:10292000FE4F4083769567958F5F6115710599F726
:1029300080E10AC020FF05C0E82FF0E0E85DFE4F0F
:102940004083369527958F5F2115310599F70895B6
:102950001F93162F9A01FA01659174910E94311DFF
:10296000AC01440F551F440F551F4E5F5F4F420F80
:10297000531F9A012E5F3F4FF90185919491FA01FF
:1029800065917491412F0E9482141F91089580E0F7
:1029900090E0FC01E45FFE4F108201968C319105BE
:1029A000C1F78091000181508093A30108958BE4C9
:1029B00087BD22E024BD25BD20936E0020936F00CB
:1029C0008DE08093810080E498E390938900809368
:1029D00088002DBB84E08093690080936800809319
:1029E0006D000895BC018530910514F465E070E038
:1029F00080E29EE40E94451D7093890060938800E8
:102A00000895AC0181E080939C0120E030E008C093
:102A10001092A1018091A1018823E1F32F5F3F4F24
:102A200024173507A8F30895EF92FF920F931F9391
:102A3000CF93DF93F82E20E030E0F901EC5BFE4FFE
:102A40008081F901E05AFE4F80832F5F3F4F2C3188
:102A5000310599F741E0EE24E39448C0C0E0D0E0AE
:102A6000DE01A85DBE4F9C91FE01EC5BFE4F8081B4
:102A70008917A0F48C913081FE01E05AFE4F20812D
:102A800090E0831B91096F2D70E00E94451D260F79
:102A900020838081FE01E458FE4F1AC09C91808102
:102AA0008E0104581E4F981788F480813C91FE01D6
:102AB000E05AFE4F208190E0831B91096F2D70E05A
:102AC0000E94451D261B2083808101C08C91F80146
:102AD00080832196CC31D10519F6E0929C011092A9
:102AE000A1018091A1018823E1F34F5FF41608F062
:102AF000B5CF20E030E0F901E85DFE4F8081F901BB
:102B0000EC5BFE4F80832F5F3F4F2C31310599F7EF
:102B1000DF91CF911F910F91FF90EF9008951F9239
:102B20000F920FB60F9211248F9381E08093A10131
:102B30008F910F900FBE0F901F9018951F920F92BC
:102B40000FB60F9211248F939F938091A3018F5FF3
:102B50008093A3019091A30180910001981708F43C
:102B600079C01092A30180919C01882309F472C05E
:102B700010929C0180917C0180930C0180917D01D9
:102B800080930D0180917E0180930E0180917F01E1
:102B900080930F01809180018093100180918101C9
:102BA00080931101809182018093120180918301B1
:102BB0008093130180918401809314018091850199
:102BC0008093150180918601809316018091870181
:102BD0008093170180918801809318018091890169
:102BE0008093190180918A0180931A0180918B0151
:102BF00080931B0180918C0180931C0180918D0139
:102C000080931D0180918E0180931E0180918F0120
:102C100080931F0180919001809320018091910108
:102C200080932101809192018093220180919301F0
:102C300080932301809194018093240180919501D8
:102C400080932501809196018093260180919701C0
:102C5000809327019091A30180911A01981710F099
:102C60005E9801C05E9A5F9A5F989091A3018091EF
:102C70001B01981710F05E9801C05E9A5F9A5F98EA
:102C80009091A30180911C01981710F05E9801C0EB
:102C90005E9A5F9A5F989091A301809120019817A6
:102CA00010F05E9801C05E9A5F9A5F989091A301C0
:102CB00080911F01981710F05E9801C05E9A5F9A8C
:102CC0005F989091A30180911E01981710F05E9873
:102CD00001C05E9A5F9A5F989091A3018091220152
:102CE000981710F05E9801C05E9A5F9A5F98909175
:102CF000A30180912101981710F05E9801C05E9A9F
:102D00005F9A5F989091A30180912301981710F02A
:102D10005E9801C05E9A5F9A5F989091A30180913E
:102D20002401981710F05E9801C05E9A5F9A5F9830
:102D30009091A30180911D01981710F05E9801C039
:102D40005E9A5F9A5F989091A301809127019817EE
:102D500010F05E9801C05E9A5F9A5F989091A3010F
:102D600080912601981710F05E9801C05E9A5F9AD4
:102D70005F989091A30180912501981710F05E98BB
:102D800001C05E9A5F9A5F985E985F9A5F985E98BE
:102D90005F9A5F989091A30180911301981710F0AA
:102DA0005E9801C05E9A5F9A5F985E985F9A5F989E
:102DB0005E985F9A5F989091A30180911601981791
:102DC00010F05E9801C05E9A5F9A5F989091A3019F
:102DD00080910F01981710F05E9801C05E9A5F9A7B
:102DE0005F989091A30180911701981710F05E9859
:102DF00001C05E9A5F9A5F989091A301809118013B
:102E0000981710F05E9801C05E9A5F9A5F98909153
:102E1000A30180911901981710F05E9801C05E9A85
:102E20005F9A5F989091A30180910C01981710F020
:102E30005E9801C05E9A5F9A5F989091A30180911D
:102E40000D01981710F05E9801C05E9A5F9A5F9826
:102E50009091A30180910E01981710F05E9801C027
:102E60005E9A5F9A5F989091A301809110019817E4
:102E700010F05E9801C05E9A5F9A5F989091A301EE
:102E800080911101981710F05E9801C05E9A5F9AC8
:102E90005F989091A30180911201981710F05E98AD
:102EA00001C05E9A5F9A5F989091A301809115018D
:102EB000981710F05E9801C05E9A5F9A5F989091A3
:102EC000A30180911401981710F05E9801C05E9ADA
:102ED0005F9A5F98299A299828989F918F910F90CF
:102EE0000FBE0F901F9018951F920F920FB60F9262
:102EF00011248F939F9391E090939F0180919E0165
:102F0000882369F4809101018F5F80930101809192
:102F10000101853011F4909301014B99FECF80910E
:102F20009E018F5F80939E0180919E01823011F4FB
:102F300010929E019F918F910F900FBE0F901F9046
:102F400018951F920F920FB60F9211248F938091B4
:102F50009D01882331F580919A018F5F80939A01BA
:102F600080919A01843011F410929A0180919A0113
:102F7000882311F48FEF11C080919A01813011F4F0
:102F800080E20BC080919A01823011F480E105C08B
:102F900080919A01833019F481E08093A2014A99CB
:102FA000FECF80919D018F5F80939D0180919D0157
:102FB000823011F410929D018F910F900FBE0F90EF
:102FC0001F90189580E090E02EEFFC01E85DFE4F29
:102FD000208301968C319105C1F7089580E090E03F
:102FE000FC01E85DFE4F108201968C319105C1F71E
:102FF0000895982F20E030E0F901E85DFE4F9083BE
:103000008091A201891718F48091A20180832F5F1B
:103010003F4F2C31310581F70895E82FF0E0E85D4E
:10302000FE4F60838091A201861718F48091A2015F
:1030300080830895FF920F931F93F82ECB016AE0CF
:1030400070E00E94451D6530710514F465E070E084
:1030500080E29EE40E94451D709389006093880081
:1030600000E062C010E020E030E0F901E85DFE4FD2
:1030700010838091A201811718F48091A2018083AE
:103080002F5F3F4F2C31310581F781E00E941415ED
:103090001F5F103441F720E030E0F901E85DFE4F9A
:1030A00010838091A201811718F48091A20180837E
:1030B0002F5F3F4F2C31310581F781E00E941415BD
:1030C0001E5F49F71FEF20E030E0F901E85DFE4F99
:1030D00010838091A201811718F48091A20180834E
:1030E0002F5F3F4F2C31310581F781E00E9414158D
:1030F00012501F3341F710E420E030E0F901E85DA1
:10310000FE4F10838091A201811718F48091A201D3
:1031100080832F5F3F4F2C31310581F781E00E9482
:103120001415115049F70F5F0F1508F49BCF1F912D
:103130000F91FF900895CF92DF92EF92FF920F933D
:103140001F937C016B010E94211DCE18DF0808949B
:10315000C11CD11CB6010E94311DE80EF91EB70139
:1031600080E090E01F910F91FF90EF90DF90CF9063
:1031700008952F923F924F925F926F927F928F921B
:103180009F92AF92BF92CF92DF92EF92FF920F93F6
:103190001F93CF93DF934C013B012A01D22EB02E17
:1031A0002E2CAC2C909303018093020168177907B1
:1031B00010F0CC2406C0861B970BBA010E94311D6B
:1031C000C62E8614970438F4C30188199909B201F0
:1031D0000E94311DC62E80910201909103016AE088
:1031E00070E00E94311D6530710514F465E070E0F7
:1031F00080E29EE40E94451D7093890060938800E0
:1032000063E370E081E090E00E949B187B0163E340
:1032100070E081E090E00E949B188B0166E070E016
:1032200081E090E00E949B18362E64E070E080E020
:1032300090E00E949B18C0E0D0E009C380E090E0DD
:10324000FC01E85DFE4F108201968C319105C1F7BB
:1032500081E0A81621F44EEF50E16D2DA1C281E06E
:10326000E816F10419F446EB51E25DC182E0E8167C
:10327000F10419F440E651E256C183E0E816F10486
:1032800019F448ED51E24FC184E0E816F10419F455
:103290004AE452E248C185E0E816F10419F444E337
:1032A00053E241C186E0E816F10419F446E653E220
:1032B0003AC187E0E816F10419F448ED53E233C14E
:1032C00088E0E816F10419F442EF55E22CC189E0D8
:1032D000E816F10419F446E654E225C18AE0E8163E
:1032E000F10419F440EB54E21EC18BE0E816F1043E
:1032F00019F44CEE57E217C18CE0E816F10419F40A
:1033000040EC56E210C18DE0E816F10419F44AE9E8
:1033100057E209C18EE0E816F10419F448E351E0E0
:1033200002C18FE0E816F10419F44AE551E0FBC050
:1033300080E1E816F10419F44CE951E0F4C081E1B0
:10334000E816F10419F442ED51E0EDC082E1E8160F
:10335000F10419F44AEA52E0E6C083E1E816F10408
:1033600019F44CE853E0DFC084E1E816F10419F4E5
:1033700042EF53E0D8C085E1E816F10419F448E3C0
:1033800056E0D1C086E1E816F10419F44AE457E0AA
:10339000CAC087E1E816F10419F440E758E0C3C059
:1033A00088E1E816F10419F44EEE59E0BCC089E159
:1033B000E816F10419F44CE75CE0B5C08AE1E816C0
:1033C000F10419F442E65DE0AEC08BE1E816F104C9
:1033D00019F440E85DE0A7C08CE1E816F10419F4A7
:1033E0004EEE5DE0A0C08DE1E816F10419F448E46A
:1033F0005EE099C08EE1E816F10419F442E25FE064
:1034000092C08FE1E816F10419F448ED5FE08BC03B
:1034100080E2E816F10419F442E850E184C081E248
:10342000E816F10419F448EC50E17DC082E2E81698
:10343000F10419F44EEF50E176C083E2E816F1048E
:1034400019F44CED51E16FC084E2E816F10419F46F
:1034500046EE52E168C085E2E816F10419F440E254
:1034600054E161C086E2E816F10419F44AED54E132
:103470005AC087E2E816F10419F448EE5CE153C043
:1034800088E2E816F10419F444E855E14CC089E2F9
:10349000E816F10419F442E950E045C08AE2E81662
:1034A000F10419F44EE856E13EC08BE2E816F1044F
:1034B00019F44CE457E137C08CE2E816F10419F432
:1034C00042E558E130C08DE2E816F10419F448EC09
:1034D00058E129C08EE2E816F10419F446E959E1F1
:1034E00022C08FE2E816F10419F44CE15AE11BC046
:1034F00080E3E816F10419F44AE05BE114C081E3CB
:10350000E816F10419F444EB5BE10DC082E3E81620
:10351000F10419F442E65CE106C083E3E816F10425
:1035200031F448E650E06D2DCE010E94A814AA2087
:1035300009F039C185E0831508F435C10130110562
:1035400019F446EB51E22BC10230110519F440E6A3
:1035500051E225C10330110519F448ED51E21FC1B4
:103560000430110519F44AE452E219C1053011057D
:1035700019F444E353E213C10630110519F446E689
:1035800053E20DC10730110519F448ED53E207C1AC
:103590000830110519F442EF55E201C10930110557
:1035A00019F446E654E2FBC00A30110519F440EB69
:1035B00054E2F5C00B30110519F44CEE57E2EFC0A0
:1035C0000C30110519F440EC56E2E9C00D3011053C
:1035D00019F44AE957E2E3C00E30110519F448E343
:1035E00051E0DDC00F30110519F44AE551E0D7C0B4
:1035F0000031110519F44CE951E0D1C00131110538
:1036000019F442ED51E0CBC00231110519F44AEA38
:1036100052E0C5C00331110519F44CE853E0BFC0B6
:103620000431110519F442EF53E0B9C00531110519
:1036300019F448E356E0B3C00631110519F44AE421
:1036400057E0ADC00731110519F440E758E0A7C0B5
:103650000831110519F44EEE59E0A1C009311105E8
:1036600019F44CE75CE09BC00A31110519F442E6FD
:103670005DE095C00B31110519F440E85DE08FC0A5
:103680000C31110519F44EEE5DE089C00D311105C4
:1036900019F448E45EE083C00E31110519F442E2EA
:1036A0005FE07DC00F31110519F448ED5FE077C090
:1036B0000032110519F442E850E171C001321105E0
:1036C00019F448EC50E16BC00232110519F44EEFC9
:1036D00050E165C00332110519F44CED51E15FC0B2
:1036E0000432110519F446EE52E159C005321105B4
:1036F00019F440E254E153C00632110519F44AEDC1
:1037000054E14DC00732110519F448EE5CE147C0A1
:103710000832110519F444E855E141C00932110598
:1037200019F442E950E03BC00A32110519F44EE8A1
:1037300056E135C00B32110519F44CE457E12FC0A6
:103740000C32110519F442E558E129C00D3211057A
:1037500019F448EC58E123C00E32110519F446E97A
:1037600059E11DC00F32110519F44CE15AE117C09F
:103770000033110519F44AE05BE111C00133110572
:1037800019F444EB5BE10BC00233110519F442E676
:103790005CE105C00333110531F448E650E06B2DC0
:1037A000CE010E94A8146814790438F480910201B3
:1037B000909103018C19910909C08614970450F463
:1037C00080910201909103018C0D911D9093030152
:1037D0008093020180910101823021F080910101EA
:1037E000833019F48DE491E014C08091010180913F
:1037F0000201909103016AE070E00E94311D653082
:10380000710514F465E070E080E29EE40E94451DBD
:10381000CB019093890080938800809101018230D0
:1038200011F48AE011C080910101833051F0809140
:103830000101843041F44AE551E26FEFCE010E946C
:10384000A81481E001C0822D0E9414152196C41590
:10385000D50508F4F3CCDF91CF911F910F91FF9024
:10386000EF90DF90CF90BF90AF909F908F907F9020
:103870006F905F904F903F902F9008954F925F927E
:103880006F927F928F929F92AF92BF92CF92EF9260
:103890000F931F9383EF84B98EEF8AB98BE487BDB2
:1038A00022E024BD25BD20936E0020936F008DE0A3
:1038B0008093810080E498E390938900809388004E
:1038C0002DBB84E0809369008093680080936D0035
:1038D00078948FEF8093A20180910201909103016F
:1038E0006AE070E00E94311D6530710514F465E0F6
:1038F00070E080E29EE40E94451D70938900609311
:10390000880081E00E941415CC24C39476E0E72E51
:1039100000E820E847E350E06CE271E08CE291E0DF
:103920000E94B9186FEF70E081E090E00E949B1850
:103930006FEF70E081E090E00E949B1869E070E01A
:1039400081E090E00E949B18E62E60E870E081E044
:1039500090E00E949B18062F60E870E081E090E004
:103960000E949B18162F6CE271E084E690E00E94A2
:103970009B182B013C0168E572E08CE291E00E940B
:103980009B184B015C0168E572E08CE291E00E94BB
:103990009B18DC01CB01CC24212FA201B401C0CFA4
:1039A000A0E0B0E0E6EDFCE10C949A1DEC01A880EB
:1039B000B980CA80DB80A114B104C104D10441F4F0
:1039C00084E2A82E89EDB82E8BE5C82E87E0D82E8C
:1039D000C601B5012DE133EF41E050E00E94771DB3
:1039E00027EA31E440E050E00E94581D7B018C0141
:1039F000C601B5012DE133EF41E050E00E94771D93
:103A0000CA01B9012CEE34EF4FEF5FEF0E94581D51
:103A10006E0D7F1D801F911F97FF04C06150704085
:103A200080409048688379838A839B839B013F779A
:103A3000C901CDB7DEB7EAE00C94B61D0E94D01CD8
:103A4000089587E091E00E94D01C0895A0E0B0E0C6
:103A50008093070190930801A0930901B0930A0194
:103A60000895AA1BBB1B51E107C0AA1FBB1FA617C5
:103A7000B70710F0A61BB70B881F991F5A95A9F717
:103A800080959095BC01CD01089597FB092E0726DE
:103A90000AD077FD04D0E5DF06D000201AF4709537
:103AA00061957F4F0895F6F7909581959F4F089502
:103AB000629FD001739FF001829FE00DF11D649F12
:103AC000E00DF11D929FF00D839FF00D749FF00D9E
:103AD000659FF00D9927729FB00DE11DF91F639F3F
:103AE000B00DE11DF91FBD01CF011124089597FB11
:103AF000092E05260ED057FD04D04BD00AD0001C4D
:103B000038F450954095309521953F4F4F4F5F4F7A
:103B10000895F6F790958095709561957F4F8F4F3A
:103B20009F4F08952F923F924F925F926F927F9294
:103B30008F929F92AF92BF92CF92DF92EF92FF92BD
:103B40000F931F93CF93DF93CDB7DEB7CA1BDB0B69
:103B50000FB6F894DEBF0FBECDBF09942A8839880E
:103B600048885F846E847D848C849B84AA84B98415
:103B7000C884DF80EE80FD800C811B81AA81B98121
:103B8000CE0FD11D0FB6F894DEBF0FBECDBFED0135
:103B90000895A1E21A2EAA1BBB1BFD010DC0AA1F8E
:103BA000BB1FEE1FFF1FA217B307E407F50720F0A6
:103BB000A21BB30BE40BF50B661F771F881F991F21
:103BC0001A9469F760957095809590959B01AC016A
:0A3BD000BD01CF010895F894FFCF66
:0C3BDA00FF012C010100FF0100000000B1
:00000001FF
